:10000000830100308A0059288C000308830199007D
:100010008B1C14288B1083120D181428031005183C
:100020000314060C8E000D140B1D5328EB308312A5
:1000300081070B11910B3F28910A2E28051A3F28A2
:100040009101910A3E28051A2C283C2810088F009F
:100050008D149101910A900192013F281208031911
:100060001E28013A0319232812080A3A03192628E0
:100070000310051A0314900C04309100920A94089E
:100080000319532814080339031D52280D1D4A284B
:1000900085154B28851183120D1113180D150314A6
:1000A0008312930C94038312190883008C0E0C0E98
:1000B00009000E308400193066200D3084000E30A7
:1000C00066208301D82B04068001840A0406031DE0
:0400D000632800346D
:1007280083128D1C942B8D100F08080083129800DB
:100738008900831608148312080808008312980099
:1007480083129408031DA42B0D111808930034304C
:100758009400080083129700B62B970A1703831298
:100768009A23A22383129603160FB12B0800831233
:10077800851594019101910A920190018D10113013
:1007880083168500FF30860083120D1095018510B1
:1007980083168112EB30831281008B160B16831699
:1007A80001178B17831208008312BB238D18EA2BBD
:1007B800F52B023096001730AE2319309600003022
:1007C800AE23F52B153083168500F52B8312942361
:1007D8003F3A0319DD2B6E3A0319E62B203A031929
:1007E800E62B83120D1CDA2B051185140E088312D3
:0807F800A2230D108510DA2B7D
:02400E00F13F80
:10420000430050005300200031002E0031002000F8
:1042100042002E00560045004C004C004500200096
:1042200028004300290032003000300034000D0027
:104230000A00200020002000200020002000200094
:10424000200020002000200020002000200020006E
:10425000200020002000200020002000200020005E
:10426000200020002000200020002000200020004E
:10427000200020002000200020002000200020003E
:00000001FF
